:03000000020026D5
:1000260075002E7500FDD2007500700000000000FE
:10003600000000000090000012009A0200AFC2000B
:10004600F5003000FDC200223000FDE500C20022AE
:10005600114E114422C3940A40023407C3343A2293
:10006600F9540F115BC9C4540F115B221166114478
:10007600C9114422C39430940A4003340322C33482
:100086000A221156117A23232323F9114E11441102
:100096007AC33922740093B40001221144A380F478
:1000A600740D1144740A11442212027F900000114B
:1000B6009A1156B461030200FEB465030200F0B45F
:1000C6006D030200E2B46C03020164B47203020120
:1000D600C1B4670612029B02026780D01156B4654E
:1000E6000302018BB469C50202281156B4650302E6
:1000F6000103B469B7020139D2000200B21188F5D2
:10010600001188F500740D1144740A1144E50011BC
:1001160072E5001172743A114474201144E0E01142
:1001260072742D11441188F0114E941B6003A38044
:10013600D401B21188F8740D1144740A1144E811FF
:1001460072743A114474201144E61172742D1144EC
:100156001188F6114E941B60030880DA01B21188EB
:10016600F5001188F5001188FB1188FAEBF9BA0041
:1001760005B9000901B21A114EF0A380F11A19113E
:100186004EF0A380E91188F5001188F5001188FA70
:1001960011A6E5001172E500117274201144114494
:1001A60074201144E01172A3E500540FB400F1E588
:1001B600009A70DC11A601B212027F12029B900017
:1001C60000119AE5701172900000119AE500117203
:1001D600900000119AE8120072900000119AE573DF
:1001E6001172900000119AEA120072900000119AA2
:1001F600EB1172900000119AEC1172900000119AA6
:10020600ED1172900000119AEE1172900000119A91
:10021600EF1172900000119AE57A1172E57B117266
:1002260001B27B007A10740D1144740A1144EB116B
:1002360072742011447420114474201144742011E6
:100246004474201144EBF8E6117274201144EB2437
:1002560001FB600BEAC39401FA70EA7A1080C701C9
:10026600B21188F5001188F500740073C200C2004F
:10027600C200D200C200C20022F5708500718872E9
:1002860089738A748B758C768D778E788F798500D5
:100296007A85007B22E570857100A872A973AA741D
:1002A600AB75AC76AD77AE78AF79857900857A0097
:0102B6002225
:00000001FF
